ARM Linker, RVCT3.1 [Build 914] for uVision [Standard]

================================================================================

Section Cross References

    startup.o(STACK) refers (Special) to stkheap2.o(.text) for __use_two_region_memory
    startup.o(HEAP) refers (Special) to stkheap2.o(.text) for __use_two_region_memory
    startup.o(RESET) refers to startup.o(STACK) for Stack_Top
    startup.o(RESET) refers to __main.o(!!!main) for __main
    startup.o(RESET) refers (Special) to stkheap2.o(.text) for __use_two_region_memory
    startup.o(.text) refers to startup.o(HEAP) for Heap_Mem
    startup.o(.text) refers to startup.o(STACK) for Stack_Mem
    startup.o(.text) refers (Special) to stkheap2.o(.text) for __use_two_region_memory
    usbhw.o(.text) refers to uwrite4.o(.text) for __aeabi_uwrite4
    usbhw.o(.text) refers to uread4.o(.text) for __aeabi_uread4
    usbhw.o(.text) refers to usbhw.o(.text) for USB_ISR
    usbhw.o(.text) refers to usbcore.o(.data) for USB_DeviceStatus
    usbhw.o(.text) refers to usbhw.o(.text) for WrCmd
    usbhw.o(.text) refers to usbuser.o(.text) for USB_Reset_Event
    usbhw.o(.text) refers to usbuser.o(.constdata) for USB_P_EP
    usbcore.o(.text) refers to usbhw.o(.text) for USB_ReadEP
    usbcore.o(.text) refers to switch8.o(.text) for __ARM_switch8
    usbcore.o(.text) refers to usbcore.o(i.USB_GetStatus) for USB_GetStatus
    usbcore.o(.text) refers to usbcore.o(i.USB_SetClrFeature) for USB_SetClrFeature
    usbcore.o(.text) refers to usbcore.o(i.USB_GetDescriptor) for USB_GetDescriptor
    usbcore.o(.text) refers to usbcore.o(i.USB_SetConfiguration) for USB_SetConfiguration
    usbcore.o(.text) refers to usbuser.o(.text) for USB_Configure_Event
    usbcore.o(.text) refers to usbcore.o(i.USB_SetInterface) for USB_SetInterface
    usbcore.o(.text) refers to mscuser.o(.text) for MSC_Reset
    usbcore.o(.text) refers to usbcore.o(.data) for USB_DeviceStatus
    usbcore.o(.text) refers to usbcore.o(.bss) for EP0Buf
    usbuser.o(.text) refers to usbcore.o(.text) for USB_ResetCore
    usbuser.o(.text) refers to mscuser.o(.text) for MSC_BulkOut
    usbuser.o(.text) refers to usbcore.o(.data) for USB_Configuration
    usbuser.o(.constdata) refers to usbcore.o(.text) for USB_EndPoint0
    usbuser.o(.constdata) refers to usbuser.o(.text) for USB_EndPoint2
    mscuser.o(.text) refers to usbhw.o(.text) for USB_WriteEP
    mscuser.o(.text) refers to uread4.o(.text) for __aeabi_uread4
    mscuser.o(.text) refers to uwrite4.o(.text) for __aeabi_uwrite4
    mscuser.o(.text) refers to mscuser.o(.data) for BulkStage
    mscuser.o(.text) refers to usbcore.o(.bss) for EP0Buf
    mscuser.o(.text) refers to mscuser.o(.bss) for Memory
    memory.o(.text) refers to usbhw.o(.text) for USB_Init
    memory.o(.text) refers to diskimg.o(.constdata) for DiskImage
    memory.o(.text) refers to mscuser.o(.bss) for Memory
    stkheap2.o(.text) refers to sys_stackheap_outer.o(.text) for __user_setup_stackheap
    stkheap2.o(.text) refers to rt_stackheap_storage_intlibspace.o(.text) for __rt_stackheap_storage
    __main.o(!!!main) refers to kernel.o(.text) for __rt_entry
    kernel.o(.text) refers to stkheap2.o(.text) for __rt_stackheap_init
    kernel.o(.text) refers to boardinit2.o(.text) for _platform_post_stackheap_init
    kernel.o(.text) refers to lib_init.o(.text) for __rt_lib_init
    kernel.o(.text) refers to boardinit3.o(.text) for _platform_post_lib_init
    kernel.o(.text) refers to exit.o(.text) for exit
    kernel.o(.text) refers to memory.o(.text) for main
    kernel.o(.text) refers to sys_exit.o(.text) for _sys_exit
    kernel.o(.ARM.exidx) refers to kernel.o(.text) for __rt_entry
    sys_stackheap_outer.o(.text) refers to libspace.o(.text) for __user_perproc_libspace
    sys_stackheap_outer.o(.text) refers to startup.o(.text) for __user_initial_stackheap
    rt_stackheap_storage.o(.text) refers to rt_stackheap_storage.o(.bss) for __rt_stackheap_storage_data
    rt_stackheap_storage_intlibspace.o(.text) refers (Weak) to libspace.o(.bss) for __libspace_start
    rt_stackheap_storage_onelibspace.o(.text) refers (Weak) to libspace.o(.text) for __user_libspace
    rt_stackheap_storage_twolibspace.o(.text) refers (Weak) to libspace.o(.text) for __user_perproc_libspace
    sys_exit.o(.text) refers to use_no_semi.o(.text) for __I_use_semihosting
    libspace.o(.text) refers to libspace.o(.bss) for __libspace_start
    exit.o(.text) refers to kernel.o(.text) for __rt_exit
    stkheap1.o(.text) refers to sys_stackheap_outer.o(.text) for __user_setup_stackheap
    stkheap1.o(.text) refers to rt_stackheap_storage_intlibspace.o(.text) for __rt_stackheap_storage
    lib_init.o(.emb_text) refers to no_argv.o(.text) for __ARM_get_argv
    lib_init.o(.text) refers to fpinit.o(x$fpl$fpinit) for _fp_init
    lib_init.o(.text) refers to lib_init.o(.emb_text) for __ARM_argv_veneer
    lib_init.o(.text) refers to rt_locale_intlibspace.o(.text) for __rt_locale
    rt_locale.o(.text) refers to rt_locale.o(.bss) for __rt_locale_data
    rt_locale_intlibspace.o(.text) refers (Weak) to libspace.o(.bss) for __libspace_start
    rt_locale_onelibspace.o(.text) refers (Weak) to libspace.o(.text) for __user_libspace
    rt_locale_twolibspace.o(.text) refers (Weak) to libspace.o(.text) for __user_perproc_libspace
    _get_argv.o(.text) refers to heapext.o(.text) for __heap_extend
    _get_argv.o(.text) refers to defsig_rtmem_outer.o(.text) for __rt_SIGRTMEM
    _get_argv.o(.text) refers to sys_command.o(.text) for _sys_command_string
    _get_argv.o(.text) refers (Special) to hrguard.o(.text) for __heap_region_guard
    fpinit.o(x$fpl$fpinit) refers to rt_fp_status_addr_intlibspace.o(.text) for __rt_fp_status_addr
    sys_command.o(.text) refers (Special) to use_no_semi.o(.text) for __I_use_semihosting
    rt_fp_status_addr.o(.text) refers to rt_fp_status_addr.o(.bss) for __rt_fp_status_addr_data
    rt_fp_status_addr_intlibspace.o(.text) refers (Weak) to libspace.o(.bss) for __libspace_start
    rt_fp_status_addr_onelibspace.o(.text) refers (Weak) to libspace.o(.text) for __user_libspace
    rt_fp_status_addr_twolibspace.o(.text) refers (Weak) to libspace.o(.text) for __user_perthread_libspace
    defsig_rtmem_outer.o(.text) refers to defsig_rtmem_inner.o(.text) for __rt_SIGRTMEM_inner
    defsig_rtmem_outer.o(.text) refers to defsig_exit.o(.text) for __sig_exit
    defsig_rtmem_formal.o(.text) refers to rt_raise.o(.text) for __rt_raise
    defsig_rtmem_formal.o(.text) refers (Special) to defsig_rtmem_inner.o(.text) for __rt_SIGRTMEM_inner
    heapext.o(.text) refers to stkheap2.o(.text) for __rt_heap_extend
    rt_raise.o(.text) refers to __raise.o(.text) for __raise
    rt_raise.o(.text) refers to sys_exit.o(.text) for _sys_exit
    defsig_exit.o(.text) refers to sys_exit.o(.text) for _sys_exit
    defsig_rtmem_inner.o(.text) refers to defsig_general.o(.text) for __default_signal_display
    __raise.o(.text) refers to defsig.o(CL$$defsig) for __default_signal_handler
    __raise.o(.text) refers to callvia.o(.text) for __ARM_call_via_r2
    defsig_general.o(.text) refers to sys_wrch.o(.text) for _ttywrch
    sys_wrch.o(.text) refers (Special) to use_no_semi.o(.text) for __I_use_semihosting
    defsig.o(CL$$defsig) refers (Weak) to defsig_rtmem_inner.o(.text) for __rt_SIGRTMEM_inner
    usbcore.o(i.USB_GetStatus) refers to usbcore.o(.text) for USB_DataInStage
    usbcore.o(i.USB_GetStatus) refers to usbcore.o(.data) for SetupPacket
    usbcore.o(i.USB_GetStatus) refers to usbcore.o(.bss) for EP0Buf
    usbcore.o(i.USB_SetClrFeature) refers to usbhw.o(.text) for USB_WakeUpCfg
    usbcore.o(i.USB_SetClrFeature) refers to usbcore.o(.data) for SetupPacket
    usbcore.o(i.USB_GetDescriptor) refers to usbcore.o(.text) for USB_DataInStage
    usbcore.o(i.USB_GetDescriptor) refers to usbcore.o(.data) for SetupPacket
    usbcore.o(i.USB_GetDescriptor) refers to usbdesc.o(.constdata) for USB_DeviceDescriptor
    usbcore.o(i.USB_SetConfiguration) refers to usbhw.o(.text) for USB_DisableEP
    usbcore.o(i.USB_SetConfiguration) refers to usbcore.o(.data) for SetupPacket
    usbcore.o(i.USB_SetConfiguration) refers to usbdesc.o(.constdata) for USB_ConfigDescriptor
    usbcore.o(i.USB_SetInterface) refers to usbhw.o(.text) for USB_ConfigEP
    usbcore.o(i.USB_SetInterface) refers to usbcore.o(.data) for USB_Configuration
    usbcore.o(i.USB_SetInterface) refers to usbdesc.o(.constdata) for USB_ConfigDescriptor


================================================================================

Adding Veneers to the image

    Adding TA veneer (8 bytes, Short) for call to '__rt_exit' from exit.o(.text).
    Adding AT veneer (12 bytes, Long) for call to '__rt_lib_shutdown' from kernel.o(.text).
    Adding AT veneer (12 bytes, Long) for call to 'USB_Resume_Event' from usbhw.o(.text).
    Adding AT veneer (12 bytes, Long) for call to 'USB_Resume' from usbhw.o(.text).
    Adding AT veneer (12 bytes, Long) for call to 'USB_Suspend_Event' from usbhw.o(.text).
    Adding AT veneer (12 bytes, Long) for call to 'USB_Suspend' from usbhw.o(.text).
    Adding AT veneer (12 bytes, Long) for call to 'USB_Reset' from usbhw.o(.text).
    Adding AT veneer (12 bytes, Long) for call to 'RdCmdDat' from usbhw.o(.text).
    Adding TA veneer (4 bytes, Inline) for call to '_fp_init' from lib_init.o(.text).
    Adding TA veneer (4 bytes, Inline) for call to '__rt_locale' from lib_init.o(.text).
    Adding AT veneer (8 bytes, Inline) for call to '__rt_lib_init' from kernel.o(.text).
    Adding TA veneer (4 bytes, Inline) for call to '__ARM_switch8' from usbcore.o(.text).
    Adding TA veneer (4 bytes, Inline) for call to '__aeabi_uwrite4' from usbhw.o(.text).
    Adding TA veneer (4 bytes, Inline) for call to '__aeabi_uread4' from usbhw.o(.text).
    Adding AT veneer (8 bytes, Inline) for call to 'USB_Reset_Event' from usbhw.o(.text).
    Adding AT veneer (8 bytes, Inline) for call to 'WrCmd' from usbhw.o(.text).
    Adding TA veneer (4 bytes, Inline) for call to '__ARM_argv_veneer' from lib_init.o(.text).

17 Veneer(s) (total 140 bytes) added to the image.

================================================================================

Image Symbol Table

    Local Symbols

    Symbol Name                              Value     Ov Type        Size  Object(Section)

    ../../angel/boardlib.s                   0x00000000   Number         0  boardinit1.o ABSOLUTE
    ../../angel/boardlib.s                   0x00000000   Number         0  boardinit3.o ABSOLUTE
    ../../angel/boardlib.s                   0x00000000   Number         0  boardinit2.o ABSOLUTE
    ../../angel/boardlib.s                   0x00000000   Number         0  boardshut.o ABSOLUTE
    ../../angel/boardlib.s                   0x00000000   Number         0  cpuinit.o ABSOLUTE
    ../../angel/handlers.s                   0x00000000   Number         0  __scatter_zi.o ABSOLUTE
    ../../angel/handlers.s                   0x00000000   Number         0  __scatter_copy.o ABSOLUTE
    ../../angel/kernel.s                     0x00000000   Number         0  kernel.o ABSOLUTE
    ../../angel/rt.s                         0x00000000   Number         0  rt_locale_twolibspace.o ABSOLUTE
    ../../angel/rt.s                         0x00000000   Number         0  rt_fp_status_addr.o ABSOLUTE
    ../../angel/rt.s                         0x00000000   Number         0  rt_fp_status_addr_twolibspace.o ABSOLUTE
    ../../angel/rt.s                         0x00000000   Number         0  rt_raise.o ABSOLUTE
    ../../angel/rt.s                         0x00000000   Number         0  rt_fp_status_addr_intlibspace.o ABSOLUTE
    ../../angel/rt.s                         0x00000000   Number         0  rt_stackheap_storage.o ABSOLUTE
    ../../angel/rt.s                         0x00000000   Number         0  rt_stackheap_storage_intlibspace.o ABSOLUTE
    ../../angel/rt.s                         0x00000000   Number         0  rt_stackheap_storage_twolibspace.o ABSOLUTE
    ../../angel/rt.s                         0x00000000   Number         0  rt_stackheap_storage_onelibspace.o ABSOLUTE
    ../../angel/rt.s                         0x00000000   Number         0  rt_fp_status_addr_onelibspace.o ABSOLUTE
    ../../angel/rt.s                         0x00000000   Number         0  rt_locale_onelibspace.o ABSOLUTE
    ../../angel/rt.s                         0x00000000   Number         0  rt_locale_intlibspace.o ABSOLUTE
    ../../angel/rt.s                         0x00000000   Number         0  rt_locale.o ABSOLUTE
    ../../angel/scatter.s                    0x00000000   Number         0  __scatter.o ABSOLUTE
    ../../angel/startup.s                    0x00000000   Number         0  __main.o ABSOLUTE
    ../../angel/sys.s                        0x00000000   Number         0  sys_stackheap_outer.o ABSOLUTE
    ../../angel/sys.s                        0x00000000   Number         0  sys_exit.o ABSOLUTE
    ../../angel/sys.s                        0x00000000   Number         0  libspace.o ABSOLUTE
    ../../angel/sys.s                        0x00000000   Number         0  use_no_semi.o ABSOLUTE
    ../../angel/sysapp.c                     0x00000000   Number         0  sys_wrch.o ABSOLUTE
    ../../angel/sysapp.c                     0x00000000   Number         0  sys_command.o ABSOLUTE
    ../../armsys.c                           0x00000000   Number         0  lib_init.o ABSOLUTE
    ../../armsys.c                           0x00000000   Number         0  lib_init.o ABSOLUTE
    ../../armsys.c                           0x00000000   Number         0  no_argv.o ABSOLUTE
    ../../armsys.c                           0x00000000   Number         0  _get_argv.o ABSOLUTE
    ../../fpinit.s                           0x00000000   Number         0  fpinit.o ABSOLUTE
    ../../heapalloc.c                        0x00000000   Number         0  hrguard.o ABSOLUTE
    ../../signal.c                           0x00000000   Number         0  defsig_rtmem_inner.o ABSOLUTE
    ../../signal.c                           0x00000000   Number         0  __raise.o ABSOLUTE
    ../../signal.c                           0x00000000   Number         0  defsig_exit.o ABSOLUTE
    ../../signal.c                           0x00000000   Number         0  defsig_general.o ABSOLUTE
    ../../signal.c                           0x00000000   Number         0  defsig_rtmem_formal.o ABSOLUTE
    ../../signal.c                           0x00000000   Number         0  defsig_rtmem_outer.o ABSOLUTE
    ../../signal.s                           0x00000000   Number         0  defsig.o ABSOLUTE
    ../../stdlib.c                           0x00000000   Number         0  exit.o ABSOLUTE
    ../../stkheap.s                          0x00000000   Number         0  heapext.o ABSOLUTE
    ../../stkheap1.s                         0x00000000   Number         0  stkheap1.o ABSOLUTE
    ../../stkheap2.s                         0x00000000   Number         0  stkheap2.o ABSOLUTE
    ../../unhosted.s                         0x00000000   Number         0  uread4.o ABSOLUTE
    ../../unhosted.s                         0x00000000   Number         0  uwrite4.o ABSOLUTE
    ../../unhosted.s                         0x00000000   Number         0  callvia.o ABSOLUTE
    ../../unhosted.s                         0x00000000   Number         0  switch8.o ABSOLUTE
    DiskImg.c                                0x00000000   Number         0  diskimg.o ABSOLUTE
    Startup.s                                0x00000000   Number         0  startup.o ABSOLUTE
    dc.s                                     0x00000000   Number         0  dc.o ABSOLUTE
    memory.c                                 0x00000000   Number         0  memory.o ABSOLUTE
    mscuser.c                                0x00000000   Number         0  mscuser.o ABSOLUTE
    usbcore.c                                0x00000000   Number         0  usbcore.o ABSOLUTE
    usbdesc.c                                0x00000000   Number         0  usbdesc.o ABSOLUTE
    usbhw.c                                  0x00000000   Number         0  usbhw.o ABSOLUTE
    usbuser.c                                0x00000000   Number         0  usbuser.o ABSOLUTE
    RESET                                    0x00002000   Section      288  startup.o(RESET)
    Undef_Handler                            0x00002040   ARM Code       4  startup.o(RESET)
    SWI_Handler                              0x00002044   ARM Code       4  startup.o(RESET)
    PAbt_Handler                             0x00002048   ARM Code       4  startup.o(RESET)
    DAbt_Handler                             0x0000204c   ARM Code       4  startup.o(RESET)
    IRQ_Handler                              0x00002050   ARM Code       4  startup.o(RESET)
    FIQ_Handler                              0x00002054   ARM Code       4  startup.o(RESET)
    !!!main                                  0x00002120   Section        8  __main.o(!!!main)
    !!!scatter                               0x00002128   Section       60  __scatter.o(!!!scatter)
    !!handler_copy                           0x00002164   Section       40  __scatter_copy.o(!!handler_copy)
    !!handler_zi                             0x0000218c   Section       44  __scatter_zi.o(!!handler_zi)
    .emb_text                                0x000021bc   Section       16  lib_init.o(.emb_text)
    .text                                    0x000021cc   Section       32  startup.o(.text)
    .text                                    0x000021f4   Section     1016  usbhw.o(.text)
    .text                                    0x000025ec   Section      416  usbhw.o(.text)
    .text                                    0x0000278c   Section      840  usbcore.o(.text)
    .text                                    0x00002adc   Section      140  usbuser.o(.text)
    .text                                    0x00002b68   Section     2040  mscuser.o(.text)
    .text                                    0x00003360   Section       60  memory.o(.text)
    .text                                    0x000033a0   Section       32  uread4.o(.text)
    .text                                    0x000033c4   Section       32  uwrite4.o(.text)
    .text                                    0x000033e4   Section       64  stkheap2.o(.text)
    .text                                    0x00003428   Section       24  switch8.o(.text)
    .text                                    0x00003440   Section      104  kernel.o(.text)
    .text                                    0x000034a8   Section       96  sys_stackheap_outer.o(.text)
    .text                                    0x00003508   Section       16  rt_stackheap_storage_intlibspace.o(.text)
    .text                                    0x00003518   Section       24  sys_exit.o(.text)
    .text                                    0x00003530   Section       12  libspace.o(.text)
    .text                                    0x0000353c   Section       12  exit.o(.text)
    .text                                    0x00003550   Section      206  lib_init.o(.text)
    .text                                    0x00003620   Section       12  boardinit2.o(.text)
    .text                                    0x0000362c   Section       16  boardinit3.o(.text)
    .text                                    0x0000363c   Section        4  use_no_semi.o(.text)
    .text                                    0x00003644   Section       16  rt_locale_intlibspace.o(.text)
    .text                                    0x00003654   Section        6  no_argv.o(.text)
    .text                                    0x0000365c   Section       16  rt_fp_status_addr_intlibspace.o(.text)
    i.USB_GetDescriptor                      0x000036c8   Section      188  usbcore.o(i.USB_GetDescriptor)
    i.USB_GetStatus                          0x00003784   Section      220  usbcore.o(i.USB_GetStatus)
    i.USB_SetClrFeature                      0x00003860   Section      232  usbcore.o(i.USB_SetClrFeature)
    i.USB_SetConfiguration                   0x00003948   Section      416  usbcore.o(i.USB_SetConfiguration)
    i.USB_SetInterface                       0x00003ae8   Section      292  usbcore.o(i.USB_SetInterface)
    x$fpl$fpinit                             0x00003c10   Section       24  fpinit.o(x$fpl$fpinit)
    .constdata                               0x00003c28   Section     4096  diskimg.o(.constdata)
    .constdata                               0x00004c28   Section      163  usbdesc.o(.constdata)
    .constdata                               0x00004ccc   Section       64  usbuser.o(.constdata)
    .data                                    0x40000000   Section       36  usbcore.o(.data)
    .data                                    0x40000024   Section       14  mscuser.o(.data)
    .bss                                     0x40000034   Section       64  usbcore.o(.bss)
    .bss                                     0x40000074   Section    16492  mscuser.o(.bss)
    .bss                                     0x400040e0   Section       96  libspace.o(.bss)
    HEAP                                     0x40004140   Number         0  startup.o(HEAP)
    STACK                                    0x40004140   Section     1288  startup.o(STACK)
    Heap_Mem                                 0x40004140   Number         0  startup.o(HEAP)
    Stack_Mem                                0x40004140   Data        1288  startup.o(STACK)
    Stack_Top                                0x40004648   Number         0  startup.o(STACK)

    Global Symbols

    Symbol Name                              Value     Ov Type        Size  Object(Section)

    BuildAttributes$$THM_ISAv1$ARM_ISAv4$M$S$PE$A:L22$X:L11$S22$IEEE1$IW$USESV6$~STKCKD$USESV7$~SHL$OSPACE$EBA8$STANDARDLIB$REQ8$EABIv2 0x00000000   Number         0  anon$$obj.o ABSOLUTE
    __ARM_use_no_argv                        0x00000000   Number         0  memory.o ABSOLUTE
    __ARM_exceptions_init                     - Undefined Weak Reference
    __Heap_DescSize                           - Undefined Weak Reference
    __alloca_initialize                       - Undefined Weak Reference
    __cpp_initialize__aeabi_                  - Undefined Weak Reference
    __cxa_finalize                            - Undefined Weak Reference
    __rt_SIGABRT_inner                        - Undefined Weak Reference
    __rt_SIGCPPL_inner                        - Undefined Weak Reference
    __rt_SIGFPE_inner                         - Undefined Weak Reference
    __rt_SIGILL_inner                         - Undefined Weak Reference
    __rt_SIGINT_inner                         - Undefined Weak Reference
    __rt_SIGPVFN_inner                        - Undefined Weak Reference
    __rt_SIGRTRED_inner                       - Undefined Weak Reference
    __rt_SIGSEGV_inner                        - Undefined Weak Reference
    __rt_SIGSTAK_inner                        - Undefined Weak Reference
    __rt_SIGTERM_inner                        - Undefined Weak Reference
    __rt_SIGUSR1_inner                        - Undefined Weak Reference
    __rt_SIGUSR2_inner                        - Undefined Weak Reference
    __rt_sigother_inner                       - Undefined Weak Reference
    __sigvec_lookup                           - Undefined Weak Reference
    __user_heap_extend                        - Undefined Weak Reference
    _atexit_init                              - Undefined Weak Reference
    _call_atexit_fns                          - Undefined Weak Reference
    _clock_init                               - Undefined Weak Reference
    _fp_trap_init                             - Undefined Weak Reference
    _get_lc_collate                           - Undefined Weak Reference
    _get_lc_ctype                             - Undefined Weak Reference
    _get_lc_monetary                          - Undefined Weak Reference
    _get_lc_numeric                           - Undefined Weak Reference
    _get_lc_time                              - Undefined Weak Reference
    _getenv_init                              - Undefined Weak Reference
    _handle_redirection                       - Undefined Weak Reference
    _init_alloc                               - Undefined Weak Reference
    _init_user_alloc                          - Undefined Weak Reference
    _initio                                   - Undefined Weak Reference
    _rand_init                                - Undefined Weak Reference
    _signal_init                              - Undefined Weak Reference
    _terminate_user_alloc                     - Undefined Weak Reference
    _terminateio                              - Undefined Weak Reference
    Reset_Handler                            0x00002058   ARM Code       0  startup.o(RESET)
    __main                                   0x00002120   ARM Code       8  __main.o(!!!main)
    __scatterload                            0x00002128   ARM Code       0  __scatter.o(!!!scatter)
    __scatterload_rt2                        0x00002128   ARM Code      52  __scatter.o(!!!scatter)
    __scatterload_null                       0x0000213c   ARM Code       0  __scatter.o(!!!scatter)
    __scatterload_copy                       0x00002164   ARM Code      40  __scatter_copy.o(!!handler_copy)
    __scatterload_zeroinit                   0x0000218c   ARM Code      44  __scatter_zi.o(!!handler_zi)
    Inline Thumb to ARM Veneer to __ARM_argv_veneer 0x000021b9   Thumb Code     0  lib_init.o(.emb_text)
    __ARM_argv_veneer                        0x000021bc   ARM Code      16  lib_init.o(.emb_text)
    __user_initial_stackheap                 0x000021cc   ARM Code       0  startup.o(.text)
    Inline ARM to Thumb Veneer to WrCmd      0x000021ec   ARM Code       0  usbhw.o(.text)
    EPAdr                                    0x000021f5   Thumb Code    16  usbhw.o(.text)
    WrCmd                                    0x00002205   Thumb Code    24  usbhw.o(.text)
    WrCmdDat                                 0x0000221d   Thumb Code    46  usbhw.o(.text)
    RdCmdDat                                 0x0000224b   Thumb Code    30  usbhw.o(.text)
    USB_SetAddress                           0x00002269   Thumb Code    50  usbhw.o(.text)
    USB_Reset                                0x0000229b   Thumb Code    52  usbhw.o(.text)
    USB_Resume                               0x000022cf   Thumb Code     2  usbhw.o(.text)
    USB_Suspend                              0x000022d1   Thumb Code     2  usbhw.o(.text)
    USB_Init                                 0x000022d3   Thumb Code   130  usbhw.o(.text)
    USB_Connect                              0x00002355   Thumb Code    34  usbhw.o(.text)
    USB_WakeUp                               0x00002377   Thumb Code    24  usbhw.o(.text)
    USB_WakeUpCfg                            0x0000238f   Thumb Code     2  usbhw.o(.text)
    USB_Configure                            0x00002391   Thumb Code    64  usbhw.o(.text)
    USB_ConfigEP                             0x000023d1   Thumb Code    74  usbhw.o(.text)
    USB_DirCtrlEP                            0x0000241b   Thumb Code     2  usbhw.o(.text)
    USB_EnableEP                             0x0000241d   Thumb Code    30  usbhw.o(.text)
    USB_DisableEP                            0x0000243b   Thumb Code    30  usbhw.o(.text)
    USB_ResetEP                              0x00002459   Thumb Code    30  usbhw.o(.text)
    USB_SetStallEP                           0x00002477   Thumb Code    30  usbhw.o(.text)
    USB_ClrStallEP                           0x00002495   Thumb Code    30  usbhw.o(.text)
    USB_ReadEP                               0x000024b3   Thumb Code   110  usbhw.o(.text)
    USB_WriteEP                              0x00002521   Thumb Code    88  usbhw.o(.text)
    USB_GetFrame                             0x00002579   Thumb Code    32  usbhw.o(.text)
    USB_ISR                                  0x000025ec   ARM Code     400  usbhw.o(.text)
    USB_ResetCore                            0x0000278d   Thumb Code    28  usbcore.o(.text)
    USB_SetupStage                           0x000027a9   Thumb Code    16  usbcore.o(.text)
    USB_DataInStage                          0x000027b9   Thumb Code    56  usbcore.o(.text)
    USB_DataOutStage                         0x000027f1   Thumb Code    38  usbcore.o(.text)
    USB_StatusInStage                        0x00002817   Thumb Code    18  usbcore.o(.text)
    USB_StatusOutStage                       0x00002829   Thumb Code    16  usbcore.o(.text)
    USB_EndPoint0                            0x00002839   Thumb Code   622  usbcore.o(.text)
    Inline ARM to Thumb Veneer to USB_Reset_Event 0x00002ad4   ARM Code       0  usbuser.o(.text)
    USB_Reset_Event                          0x00002add   Thumb Code    20  usbuser.o(.text)
    USB_Suspend_Event                        0x00002af1   Thumb Code    10  usbuser.o(.text)
    USB_Resume_Event                         0x00002afb   Thumb Code    10  usbuser.o(.text)
    USB_Configure_Event                      0x00002b05   Thumb Code    28  usbuser.o(.text)
    USB_EndPoint1                            0x00002b21   Thumb Code     2  usbuser.o(.text)
    USB_EndPoint2                            0x00002b23   Thumb Code    34  usbuser.o(.text)
    USB_EndPoint3                            0x00002b45   Thumb Code     2  usbuser.o(.text)
    USB_EndPoint4                            0x00002b47   Thumb Code     2  usbuser.o(.text)
    USB_EndPoint5                            0x00002b49   Thumb Code     2  usbuser.o(.text)
    USB_EndPoint6                            0x00002b4b   Thumb Code     2  usbuser.o(.text)
    USB_EndPoint7                            0x00002b4d   Thumb Code     2  usbuser.o(.text)
    USB_EndPoint8                            0x00002b4f   Thumb Code     2  usbuser.o(.text)
    USB_EndPoint9                            0x00002b51   Thumb Code     2  usbuser.o(.text)
    USB_EndPoint10                           0x00002b53   Thumb Code     2  usbuser.o(.text)
    USB_EndPoint11                           0x00002b55   Thumb Code     2  usbuser.o(.text)
    USB_EndPoint12                           0x00002b57   Thumb Code     2  usbuser.o(.text)
    USB_EndPoint13                           0x00002b59   Thumb Code     2  usbuser.o(.text)
    USB_EndPoint14                           0x00002b5b   Thumb Code     2  usbuser.o(.text)
    USB_EndPoint15                           0x00002b5d   Thumb Code     2  usbuser.o(.text)
    MSC_Reset                                0x00002b69   Thumb Code    18  mscuser.o(.text)
    MSC_GetMaxLUN                            0x00002b7b   Thumb Code    10  mscuser.o(.text)
    MSC_MemoryRead                           0x00002b85   Thumb Code   144  mscuser.o(.text)
    MSC_SetCSW                               0x00002c15   Thumb Code    36  mscuser.o(.text)
    MSC_MemoryWrite                          0x00002c39   Thumb Code   162  mscuser.o(.text)
    MSC_MemoryVerify                         0x00002cdb   Thumb Code   180  mscuser.o(.text)
    MSC_RWSetup                              0x00002d8f   Thumb Code   110  mscuser.o(.text)
    DataInFormat                             0x00002dfd   Thumb Code    70  mscuser.o(.text)
    DataInTransfer                           0x00002e43   Thumb Code    82  mscuser.o(.text)
    MSC_TestUnitReady                        0x00002e95   Thumb Code    56  mscuser.o(.text)
    MSC_RequestSense                         0x00002ecd   Thumb Code    84  mscuser.o(.text)
    MSC_Inquiry                              0x00002f21   Thumb Code   212  mscuser.o(.text)
    MSC_ModeSense6                           0x00002ff5   Thumb Code    44  mscuser.o(.text)
    MSC_ModeSense10                          0x00003021   Thumb Code    54  mscuser.o(.text)
    MSC_ReadCapacity                         0x00003057   Thumb Code    58  mscuser.o(.text)
    MSC_ReadFormatCapacity                   0x00003091   Thumb Code    72  mscuser.o(.text)
    MSC_GetCBW                               0x000030d9   Thumb Code   444  mscuser.o(.text)
    MSC_BulkIn                               0x00003295   Thumb Code    76  mscuser.o(.text)
    MSC_BulkOut                              0x000032e1   Thumb Code    94  mscuser.o(.text)
    main                                     0x00003361   Thumb Code    46  memory.o(.text)
    Inline Thumb to ARM Veneer to __aeabi_uread4 0x0000339d   Thumb Code     0  uread4.o(.text)
    __aeabi_uread4                           0x000033a0   ARM Code       0  uread4.o(.text)
    __rt_uread4                              0x000033a0   ARM Code      32  uread4.o(.text)
    Inline Thumb to ARM Veneer to __aeabi_uwrite4 0x000033c1   Thumb Code     0  uwrite4.o(.text)
    __aeabi_uwrite4                          0x000033c4   ARM Code       0  uwrite4.o(.text)
    __rt_uwrite4                             0x000033c4   ARM Code      32  uwrite4.o(.text)
    __use_two_region_memory                  0x000033e4   ARM Code       4  stkheap2.o(.text)
    __rt_stackheap_init                      0x000033e8   ARM Code      36  stkheap2.o(.text)
    __rt_heap_extend                         0x0000340c   ARM Code      24  stkheap2.o(.text)
    Inline Thumb to ARM Veneer to __ARM_switch8 0x00003425   Thumb Code     0  switch8.o(.text)
    __ARM_switch8                            0x00003428   ARM Code      24  switch8.o(.text)
    __rt_switch8                             0x00003428   ARM Code       0  switch8.o(.text)
    __rt_entry                               0x00003440   ARM Code      76  kernel.o(.text)
    __rt_exit                                0x0000348c   ARM Code      20  kernel.o(.text)
    __rt_abort                               0x000034a0   ARM Code       8  kernel.o(.text)
    __user_setup_stackheap                   0x000034a8   ARM Code      96  sys_stackheap_outer.o(.text)
    __rt_stackheap_storage                   0x00003508   ARM Code      12  rt_stackheap_storage_intlibspace.o(.text)
    _sys_exit                                0x00003518   ARM Code      20  sys_exit.o(.text)
    __user_libspace                          0x00003530   ARM Code       8  libspace.o(.text)
    __user_perproc_libspace                  0x00003530   ARM Code       0  libspace.o(.text)
    __user_perthread_libspace                0x00003530   ARM Code       0  libspace.o(.text)
    exit                                     0x0000353d   Thumb Code    12  exit.o(.text)
    Inline ARM to Thumb Veneer to __rt_lib_init 0x00003548   ARM Code       0  lib_init.o(.text)
    __rt_lib_init                            0x00003551   Thumb Code   184  lib_init.o(.text)
    __rt_lib_shutdown                        0x00003609   Thumb Code    22  lib_init.o(.text)
    _platform_post_stackheap_init            0x00003620   ARM Code      12  boardinit2.o(.text)
    _platform_post_lib_init                  0x0000362c   ARM Code      16  boardinit3.o(.text)
    __I_use_semihosting                      0x0000363c   ARM Code       0  use_no_semi.o(.text)
    __use_no_semihosting_swi                 0x0000363c   ARM Code       4  use_no_semi.o(.text)
    Inline Thumb to ARM Veneer to __rt_locale 0x00003641   Thumb Code     0  rt_locale_intlibspace.o(.text)
    __rt_locale                              0x00003644   ARM Code      12  rt_locale_intlibspace.o(.text)
    __ARM_get_argv                           0x00003655   Thumb Code     6  no_argv.o(.text)
    __rt_fp_status_addr                      0x0000365c   ARM Code      12  rt_fp_status_addr_intlibspace.o(.text)
    Long ARM to Thumb Veneer to RdCmdDat     0x0000366c   ARM Code       0  anon$$obj.o(Veneer$$Code)
    Long ARM to Thumb Veneer to USB_Reset    0x00003678   ARM Code       0  anon$$obj.o(Veneer$$Code)
    Long ARM to Thumb Veneer to USB_Suspend  0x00003684   ARM Code       0  anon$$obj.o(Veneer$$Code)
    Long ARM to Thumb Veneer to USB_Suspend_Event 0x00003690   ARM Code       0  anon$$obj.o(Veneer$$Code)
    Long ARM to Thumb Veneer to USB_Resume   0x0000369c   ARM Code       0  anon$$obj.o(Veneer$$Code)
    Long ARM to Thumb Veneer to USB_Resume_Event 0x000036a8   ARM Code       0  anon$$obj.o(Veneer$$Code)
    Long ARM to Thumb Veneer to __rt_lib_shutdown 0x000036b4   ARM Code       0  anon$$obj.o(Veneer$$Code)
    Short Thumb to ARM Veneer to __rt_exit   0x000036c1   Thumb Code     0  anon$$obj.o(Veneer$$Code)
    USB_GetDescriptor                        0x000036c9   Thumb Code   166  usbcore.o(i.USB_GetDescriptor)
    USB_GetStatus                            0x00003785   Thumb Code   188  usbcore.o(i.USB_GetStatus)
    USB_SetClrFeature                        0x00003861   Thumb Code   212  usbcore.o(i.USB_SetClrFeature)
    USB_SetConfiguration                     0x00003949   Thumb Code   380  usbcore.o(i.USB_SetConfiguration)
    USB_SetInterface                         0x00003ae9   Thumb Code   268  usbcore.o(i.USB_SetInterface)
    Inline Thumb to ARM Veneer to _fp_init   0x00003c0d   Thumb Code     0  fpinit.o(x$fpl$fpinit)
    _fp_init                                 0x00003c10   ARM Code      24  fpinit.o(x$fpl$fpinit)
    __fplib_config_pureend_doubles           0x00003c20   ARM Code       0  fpinit.o(x$fpl$fpinit)
    DiskImage                                0x00003c28   Data        4096  diskimg.o(.constdata)
    USB_DeviceDescriptor                     0x00004c28   Data          18  usbdesc.o(.constdata)
    USB_ConfigDescriptor                     0x00004c3a   Data          33  usbdesc.o(.constdata)
    USB_StringDescriptor                     0x00004c5b   Data         112  usbdesc.o(.constdata)
    USB_P_EP                                 0x00004ccc   Data          64  usbuser.o(.constdata)
    Region$$Table$$Base                      0x00004d0c   Number         0  anon$$obj.o(Region$$Table)
    Region$$Table$$Limit                     0x00004d2c   Number         0  anon$$obj.o(Region$$Table)
    USB_DeviceStatus                         0x40000000   Data           2  usbcore.o(.data)
    USB_DeviceAddress                        0x40000002   Data           1  usbcore.o(.data)
    USB_Configuration                        0x40000003   Data           1  usbcore.o(.data)
    USB_EndPointMask                         0x40000004   Data           4  usbcore.o(.data)
    USB_EndPointHalt                         0x40000008   Data           4  usbcore.o(.data)
    USB_NumInterfaces                        0x4000000c   Data           1  usbcore.o(.data)
    USB_AltSetting                           0x4000000d   Data           4  usbcore.o(.data)
    EP0Data                                  0x40000014   Data           8  usbcore.o(.data)
    SetupPacket                              0x4000001c   Data           8  usbcore.o(.data)
    MemOK                                    0x40000024   Data           4  mscuser.o(.data)
    Offset                                   0x40000028   Data           4  mscuser.o(.data)
    Length                                   0x4000002c   Data           4  mscuser.o(.data)
    BulkStage                                0x40000030   Data           1  mscuser.o(.data)
    BulkLen                                  0x40000031   Data           1  mscuser.o(.data)
    EP0Buf                                   0x40000034   Data          64  usbcore.o(.bss)
    Memory                                   0x40000074   Data       16384  mscuser.o(.bss)
    BulkBuf                                  0x40004074   Data          64  mscuser.o(.bss)
    CBW                                      0x400040b4   Data          31  mscuser.o(.bss)
    CSW                                      0x400040d3   Data          13  mscuser.o(.bss)
    __libspace_start                         0x400040e0   Data          96  libspace.o(.bss)
    __temporary_stack_top_libspace           0x40004140   Data           0  libspace.o(.bss)


================================================================================

Memory Map of the image

  Image Entry point : 0x00002000

  Load Region LR_IROM1 (Base: 0x00002000, Size: 0x00002d60, Max: 0x00080000, ABSOLUTE)

    Execution Region ER_IROM1 (Base: 0x00002000, Size: 0x00002d2c, Max: 0x00080000, ABSOLUTE)

    Base Addr    Size         Type   Attr      Idx    E Section Name        Object

    0x00002000   0x00000120   Code   RO            3  * RESET               startup.o
    0x00002120   0x00000008   Code   RO          241  * !!!main             __main.o(c_t.l)
    0x00002128   0x0000003c   Code   RO          334    !!!scatter          __scatter.o(c_t.l)
    0x00002164   0x00000028   Code   RO          336    !!handler_copy      __scatter_copy.o(c_t.l)
    0x0000218c   0x0000002c   Code   RO          338    !!handler_zi        __scatter_zi.o(c_t.l)
    0x000021b8   0x00000004   Ven    RO          268    .emb_text           lib_init.o(c_t.l)
    0x000021bc   0x00000010   Code   RO          268    .emb_text           lib_init.o(c_t.l)
    0x000021cc   0x00000020   Code   RO            4    .text               startup.o
    0x000021ec   0x00000008   Ven    RO           29    .text               usbhw.o
    0x000021f4   0x000003f8   Code   RO           29    .text               usbhw.o
    0x000025ec   0x000001a0   Code   RO           30    .text               usbhw.o
    0x0000278c   0x00000348   Code   RO           75    .text               usbcore.o
    0x00002ad4   0x00000008   Ven    RO          173    .text               usbuser.o
    0x00002adc   0x0000008c   Code   RO          173    .text               usbuser.o
    0x00002b68   0x000007f8   Code   RO          201    .text               mscuser.o
    0x00003360   0x0000003c   Code   RO          219    .text               memory.o
    0x0000339c   0x00000004   Ven    RO          235    .text               uread4.o(c_t.l)
    0x000033a0   0x00000020   Code   RO          235    .text               uread4.o(c_t.l)
    0x000033c0   0x00000004   Ven    RO          237    .text               uwrite4.o(c_t.l)
    0x000033c4   0x00000020   Code   RO          237    .text               uwrite4.o(c_t.l)
    0x000033e4   0x00000040   Code   RO          239    .text               stkheap2.o(c_t.l)
    0x00003424   0x00000004   Ven    RO          243    .text               switch8.o(h_t.l)
    0x00003428   0x00000018   Code   RO          243    .text               switch8.o(h_t.l)
    0x00003440   0x00000068   Code   RO          245    .text               kernel.o(c_t.l)
    0x000034a8   0x00000060   Code   RO          248    .text               sys_stackheap_outer.o(c_t.l)
    0x00003508   0x00000010   Code   RO          253    .text               rt_stackheap_storage_intlibspace.o(c_t.l)
    0x00003518   0x00000018   Code   RO          259    .text               sys_exit.o(c_t.l)
    0x00003530   0x0000000c   Code   RO          261    .text               libspace.o(c_t.l)
    0x0000353c   0x0000000c   Code   RO          264    .text               exit.o(c_t.l)
    0x00003548   0x00000008   Ven    RO          269    .text               lib_init.o(c_t.l)
    0x00003550   0x000000ce   Code   RO          269    .text               lib_init.o(c_t.l)
    0x0000361e   0x00000002   PAD
    0x00003620   0x0000000c   Code   RO          274    .text               boardinit2.o(c_t.l)
    0x0000362c   0x00000010   Code   RO          276    .text               boardinit3.o(c_t.l)
    0x0000363c   0x00000004   Code   RO          280    .text               use_no_semi.o(c_t.l)
    0x00003640   0x00000004   Ven    RO          285    .text               rt_locale_intlibspace.o(c_t.l)
    0x00003644   0x00000010   Code   RO          285    .text               rt_locale_intlibspace.o(c_t.l)
    0x00003654   0x00000006   Code   RO          295    .text               no_argv.o(c_t.l)
    0x0000365a   0x00000002   PAD
    0x0000365c   0x00000010   Code   RO          304    .text               rt_fp_status_addr_intlibspace.o(c_t.l)
    0x0000366c   0x0000000c   Ven    RO          349    Veneer$$Code        anon$$obj.o
    0x00003678   0x0000000c   Ven    RO          350    Veneer$$Code        anon$$obj.o
    0x00003684   0x0000000c   Ven    RO          351    Veneer$$Code        anon$$obj.o
    0x00003690   0x0000000c   Ven    RO          352    Veneer$$Code        anon$$obj.o
    0x0000369c   0x0000000c   Ven    RO          353    Veneer$$Code        anon$$obj.o
    0x000036a8   0x0000000c   Ven    RO          354    Veneer$$Code        anon$$obj.o
    0x000036b4   0x0000000c   Ven    RO          355    Veneer$$Code        anon$$obj.o
    0x000036c0   0x00000008   Ven    RO          356    Veneer$$Code        anon$$obj.o
    0x000036c8   0x000000bc   Code   RO          101    i.USB_GetDescriptor  usbcore.o
    0x00003784   0x000000dc   Code   RO           87    i.USB_GetStatus     usbcore.o
    0x00003860   0x000000e8   Code   RO           94    i.USB_SetClrFeature  usbcore.o
    0x00003948   0x000001a0   Code   RO          108    i.USB_SetConfiguration  usbcore.o
    0x00003ae8   0x00000124   Code   RO          115    i.USB_SetInterface  usbcore.o
    0x00003c0c   0x00000004   Ven    RO          297    x$fpl$fpinit        fpinit.o(fz_ts.l)
    0x00003c10   0x00000018   Code   RO          297    x$fpl$fpinit        fpinit.o(fz_ts.l)
    0x00003c28   0x00001000   Data   RO           12    .constdata          diskimg.o
    0x00004c28   0x000000a3   Data   RO          151    .constdata          usbdesc.o
    0x00004ccb   0x00000001   PAD
    0x00004ccc   0x00000040   Data   RO          174    .constdata          usbuser.o
    0x00004d0c   0x00000020   Data   RO          333    Region$$Table       anon$$obj.o


    Execution Region RW_IRAM1 (Base: 0x40000000, Size: 0x00004648, Max: 0x00008000, ABSOLUTE)

    Base Addr    Size         Type   Attr      Idx    E Section Name        Object

    0x40000000   0x00000024   Data   RW           76    .data               usbcore.o
    0x40000024   0x0000000e   Data   RW          202    .data               mscuser.o
    0x40000032   0x00000002   PAD
    0x40000034   0x00000040   Zero   RW           77    .bss                usbcore.o
    0x40000074   0x0000406c   Zero   RW          203    .bss                mscuser.o
    0x400040e0   0x00000060   Zero   RW          262    .bss                libspace.o(c_t.l)
    0x40004140   0x00000000   Zero   RW            2    HEAP                startup.o
    0x40004140   0x00000508   Zero   RW            1    STACK               startup.o


================================================================================

Image component sizes


      Code (inc. data)   RO Data    RW Data    ZI Data      Debug   Object Name

         0          0       4096          0          0       1932   diskimg.o
        60         14          0          0          0        415   memory.o
      2040         82          0         14      16492       6084   mscuser.o
       320         64          0          0       1288        452   startup.o
      2188        204          0         36         64      11253   usbcore.o
         0          0        163          0          0       1017   usbdesc.o
      1432        100          0          0          0      12480   usbhw.o
       140         10         64          0          0       2906   usbuser.o

    ------------------------------------------------------------------------
      6288        502       4356         52      17844      36540   Object Totals
       108         28         32          0          0          0   (incl. Generated)
         0          0          1          2          0          1   (incl. Padding)

    ------------------------------------------------------------------------

      Code (inc. data)   RO Data    RW Data    ZI Data      Debug   Library Member Name

         8          0          0          0          0          0   __main.o
        60          8          0          0          0          0   __scatter.o
        40          0          0          0          0          0   __scatter_copy.o
        44          0          0          0          0          0   __scatter_zi.o
        12          0          0          0          0          0   boardinit2.o
        16          0          0          0          0          0   boardinit3.o
        12          0          0          0          0          0   exit.o
        28          0          0          0          0          0   fpinit.o
       104          4          0          0          0          0   kernel.o
       234          4          0          0          0          0   lib_init.o
        12          4          0          0         96          0   libspace.o
         6          0          0          0          0          0   no_argv.o
        16          4          0          0          0          0   rt_fp_status_addr_intlibspace.o
        20          4          0          0          0          0   rt_locale_intlibspace.o
        16          4          0          0          0          0   rt_stackheap_storage_intlibspace.o
        64          0          0          0          0          0   stkheap2.o
        28          0          0          0          0          0   switch8.o
        24          8          0          0          0          0   sys_exit.o
        96          0          0          0          0          0   sys_stackheap_outer.o
        36          0          0          0          0          0   uread4.o
         4          0          0          0          0          0   use_no_semi.o
        36          0          0          0          0          0   uwrite4.o

    ------------------------------------------------------------------------
       920         40          0          0         96          0   Library Totals
         4          0          0          0          0          0   (incl. Padding)

    ------------------------------------------------------------------------

      Code (inc. data)   RO Data    RW Data    ZI Data      Debug   Library Name

       860         40          0          0         96          0   c_t.l
        28          0          0          0          0          0   fz_ts.l
        28          0          0          0          0          0   h_t.l

    ------------------------------------------------------------------------
       920         40          0          0         96          0   Library Totals

    ------------------------------------------------------------------------

================================================================================


      Code (inc. data)   RO Data    RW Data    ZI Data      Debug   

      7208        542       4356         52      17940      36540   Grand Totals
      7208        542       4356         52      17940      36540   ELF Image Totals
      7208        542       4356         52          0          0   ROM Totals

================================================================================

    Total RO  Size (Code + RO Data)                11564 (  11.29kB)
    Total RW  Size (RW Data + ZI Data)             17992 (  17.57kB)
    Total ROM Size (Code + RO Data + RW Data)      11616 (  11.34kB)

================================================================================

